:100000000C9462050C94A9050C94A9050C94A905FF
:100010000C94A9050C94A9050C94A9050C94A905A8
:100020000C94A9050C94A9050C94590F0C942B1051
:100030000C948F1E0C94A9050C94A9050C94A90589
:100040000C94A9050C94A9050C94A9050C94A90578
:100050000C94A9050C94031F0C94A9050C94A905F4
:100060000C94A9050C94A9050C94A9050C94A90558
:100070000C94A9050C94A9050C94A9050C94A90548
:100080000C94A9050C94A9050C94A9050C94A90538
:100090000C94A9050C94A9050C94A9050C94A90528
:1000A0000C94A9050C94A9050C94A9059810BA10F4
:1000B000A811BA10A811FF102211A81177118A11E6
:1000C0004615461574157415D1150F1628182818DD
:1000D0002816281829172917FC1728182818131864
:1000E000041607090B0A1D1B06196405141A0815C6
:1000F0001C171E1F202123222E26242D25273012D7
:10010000182F0C13280F0D340E33313638111037D9
:100110002B2C352A5829787B79397A504F515272D5
:100120006C63685680668053020103555880576D92
:100130006E5462595A5B5C5D5E5F6F606174756698
:100140003E3F403C4142774476466B47804365459D
:100150008048494A4B4C3D4D3B4E3A7D7E7C7F73F7
:100160006164625F686F73745F6B62645F72656322
:10017000763A204552524F52282564290A000A0037
:1001800025303458006164625F686F73745F6B621E
:10019000645F726563763A20004552524F523A20AE
:1001A0006D65646961206B6579300A004552524F74
:1001B000523A206D65646961206B6579310A005D92
:1001C0000A0025640020002564007C002530325898
:1001D00000200025303258006164625F6D6F7573D6
:1001E00065207261773A205B000A00253031366263
:1001F000006164625F686F73745F6D6F7573655FD4
:10020000726563763A2000646562756720656E6189
:10021000626C65642E0A005363616E3A2061646407
:10022000723A25642C20726567333A253034580AB7
:1002300000416674657220696E69743A0A00466FFF
:10024000756E643A206D65646961206B6579730A27
:10025000005363616E3A20616464723A25642C2015
:10026000726567333A253034580A004265666F720A
:100270006520696E69743A0A004B6579626F617234
:10028000642073746172742E0A0055534220636FA8
:100290006E666967757265642E0A000D0A696E697B
:1002A000740A005B445D005B435D002E0341004423
:1002B00000420020006B006500790062006F006161
:1002C0000072006400200063006F006E007600651D
:1002D00000720074006500720000000E0374002EAE
:1002E000006D002E006B002E0000000403090409BD
:1002F000027400040100A03209040000010301019E
:1003000000092111010001224000070581030800B6
:100310000A09040100010301020009211101000181
:10032000224D000705820308000A090402000103A8
:100330000000000921110100012236000705830396
:1003400008000A090403000203000000092111014A
:100350000001222200070584032000010705040391
:100360002000011201100100000008EDFEDB0A016F
:1003700001010200010631FF0974A1010975150090
:1003800026FF009520750881020976150026FF00DA
:10039000952075089102C005010980A1018502160A
:1003A000810026B7001A81002AB7007510950181D7
:1003B00000C0050C0901A1018503160100269C025D
:1003C0001A01002A9C02751095018100C0050109DF
:1003D00002A1010901A1000509190129051500253E
:1003E00001950575018102950175038101050109DA
:1003F0003009311581257F95027508810609381568
:1004000081257F950175088106050C0A3802158142
:10041000257F950175088106C0C005010906A10167
:10042000050719E029E715002501950875018102E6
:1004300095017508810105081901290595057501C2
:1004400091029501750391010507190029FF150017
:1004500026FF00950675088100C0636F6E73756D89
:1004600065723A20253034580A0073797374656DCB
:100470003A20253034580A000A002530325820002E
:100480006B6579626F6172643A20004C45443A2092
:10049000253032580A00253032583A20253038624B
:1004A00025730A00722F63203031323334353637EA
:1004B0000A00290A002575002F002575005D280017
:1004C000256400200025640020002564002000250C
:1004D00064007C0025303258006D6F7573656B6564
:1004E00079205B62746E7C782079207620685D28A4
:1004F0007265702F61636C293A205B006D6B5F77CA
:100500006865656C5F74696D655F746F5F6D617858
:10051000203D2025640A006D6B5F776865656C5F20
:100520006D61785F7370656564203D2025640A0005
:100530006D6B5F74696D655F746F5F6D6178203D91
:100540002025640A006D6B5F6D61785F737065656F
:1005500064203D2025640A006D6B5F696E746572CE
:1005600076616C203D2025640A006D6B5F64656CCC
:100570006179203D2025640A006D6B5F77686565B1
:100580006C5F74696D655F746F5F6D6178203D208D
:1005900025640A006D6B5F776865656C5F6D6178D7
:1005A0005F7370656564203D2025640A006D6B5F94
:1005B00074696D655F746F5F6D6178203D2025649F
:1005C0000A006D6B5F6D61785F7370656564203DD7
:1005D0002025640A006D6B5F696E74657276616CCC
:1005E000203D2025640A006D6B5F64656C61792095
:1005F0003D2025640A000A00257500363A207768F8
:1006000065656C5F74696D655F746F5F6D61783A85
:1006100020000A00257500353A20776865656C5F13
:100620006D61785F73706565643A20000A00257516
:1006300000343A2074696D655F746F5F6D61783A5C
:1006400020000A00257500333A206D61785F7370D1
:100650006565643A20000A00257500323A20696E0B
:1006600074657276616C286D73293A20000A002542
:100670007500313A2064656C6179282A31306D73D8
:10068000293A20000A092D2056616C756573202DCA
:100690000A004D3E004D25643E20003F0073657406
:1006A0002064656661756C740A00433E20007768BB
:1006B0006572652064656C74613A20637572736F4E
:1006C000723D25642C20776865656C3D25640A536E
:1006D000656520687474703A2F2F656E2E77696B8C
:1006E0006970656469612E6F72672F77696B692F16
:1006F0004D6F7573655F6B6579730A000A092D206C
:100700004D6F7573656B6579202D0A4553432F71C5
:100710003A09717569740A313A0964656C6179281E
:100720002A31306D73290A323A09696E746572761E
:10073000616C286D73290A333A096D61785F7370B3
:100740006565640A343A0974696D655F746F5F6D3D
:1007500061780A353A09776865656C5F6D61785F25
:1007600073706565640A363A09776865656C5F740D
:10077000696D655F746F5F6D61780A0A703A097020
:1007800072696E742076616C7565730A643A0973D8
:1007900065742064656661756C74730A75703A09D6
:1007A0002B310A646F776E3A092D310A70677570C4
:1007B0003A092B31300A7067646F776E3A092D3130
:1007C000300A0A7370656564203D2064656C74614D
:1007D000202A206D61785F7370656564202A202867
:1007E000726570656174202F2074696D655F746F28
:1007F0005F6D6178290A003F004D3E2000433E2096
:10080000004C25640A000A092D20436F6E736F6C3B
:1008100065202D0A4553432F713A09717569740A91
:100820006D3A096D6F7573656B65790A000A092D5C
:10083000204D61676963202D0A643A096465627519
:10084000670A783A096465627567206D6174726938
:10085000780A6B3A096465627567206B6579626F27
:100860006172640A6D3A096465627567206D6F751F
:1008700073650A763A0976657273696F6E0A733A20
:10088000097374617475730A633A09636F6E736FE9
:100890006C65206D6F64650A302D343A096C61799E
:1008A0006572302D34284631302D4634290A506186
:1008B00075733A09626F6F746C6F616465720A00D8
:1008C0003F0074696D65725F726561643332282917
:1008D0003A202530346C580A006B6579626F61727A
:1008E000645F69646C653A2025580A006B6579621B
:1008F0006F6172645F70726F746F636F6C3A202502
:10090000580A00686F73745F6B6579626F61726417
:100910005F6C65647328293A2025580A000A092D5E
:1009200020537461747573202D0A004743433A20A5
:10093000342E392E32204156522D4C4942433A2012
:10094000312E382E3073766E204156525F4152431D
:10095000483A20617672350A004F5054494F4E5341
:100960003A204C554641204D4F5553454B45592053
:1009700045585452414B455920434F4E534F4C45D7
:1009800020434F4D4D414E44204B45594D41505F02
:1009900053454354494F4E20343039360A004255AE
:1009A000494C443A20353330383138622D6469720D
:1009B0007479202831353A35323A3231204A616E25
:1009C0002031342032303137290A005649443A2048
:1009D00030784645454428742E6D2E6B2E292050C4
:1009E00049443A2030783041444228414442206B07
:1009F0006579626F61726420636F6E76657274658B
:100A00007229205645523A203078303130310A0070
:100A1000444553433A20636F6E76657274204144B7
:100A200042206B6579626F61726420746F20555348
:100A3000420A000A092D2056657273696F6E202DD7
:100A40000A000A6D6F7573653A206F66660A000AC0
:100A50006D6F7573653A206F6E0A000A6B65796277
:100A60006F6172643A206F66660A000A6B6579628C
:100A70006F6172643A206F6E0A000A6D6174726968
:100A8000783A206F66660A000A6D61747269783A76
:100A9000206F6E0A000A64656275673A206F6E0AFD
:100AA000000A64656275673A206F66660A000A0A82
:100AB000626F6F746C6F616465722E2E2E2000431E
:100AC0003E20000011241FBECFEFDAE0DEBFCDBF15
:100AD00004B603FE27C08091DC019091DD01A09156
:100AE000DE01B091DF018730904BA740B04BD1F4CD
:100AF0001092DC011092DD011092DE011092DF01F4
:100B000014BE84B7877F84BF0FB6F894A8958091F0
:100B10006000886180936000109260000FBEE0E08A
:100B2000F8E3099511E0A0E0B1E0E8EDFEE402C0D1
:100B300005900D92A433B107D9F721E0A4E3B1E009
:100B400001C01D92AC3DB207E1F70E94870C0C94E6
:100B50006A270C940000FF93EF93E0913401F09129
:100B60003501309709F00995EF91FF910895FC0147
:100B70008591803011F0EFDFFBCF0895FF27E0E291
:100B800030E247FF0CC0419597FF09C0EDE2609548
:100B9000709580959095611D711D811D911D27FF98
:100BA00002C0219530E350E2AA27660F771F881F05
:100BB000991FAA1FA41710F0A41B63955A95A9F7B3
:100BC000AA3008F0A95FA05DAF93F3956115710598
:100BD0008105910541F7ED3211F4EF93F395F2178A
:100BE00018F43F93F395FBCF8F91B5DFFA95E1F7BA
:100BF0000895E991F9918591803021F0853219F0BD
:100C0000AADFF9CF089520E0E89455915532C1F359
:100C1000503311F4689455915A3348F4505390F37B
:100C2000220F022E220F220F200D250FF4CF0EF4DB
:100C3000219589919991533619F3533729F15335F9
:100C400059F1BC0188279927E8945C3621F48991F1
:100C5000999168945591543639F446EF7EF077FFB8
:100C60000DC08FEF9FEF0AC055374AE039F0583575
:100C700040E121F0523642E009F00895FF93EF93EE
:100C80007DDFEF91FF91B7CFFF93EF93FC0181914F
:100C90008030B9F360DFFBCFFF93EF9368DFF1CFD4
:100CA000DF93CF93CDB7DEB72596A3DFCF91DF914A
:100CB0000895282F2770E82FE695E695E695EF70C2
:100CC000F0E0E95CFE4F87FF0AC081E090E001C0E0
:100CD000880F2A95EAF780959081892308C081E0E2
:100CE00090E001C0880F2A95EAF79081892B8083D4
:100CF00008950F931F93CF93DF93569A5E9A0E94A5
:100D000066092FEF87EA91E6215080409040E1F795
:100D100000C000008BE692E09F938F930E945006E4
:100D20000F900F90C1E0D0E001E512E063E08C2F5E
:100D30000E946A09009771F09F938F93DF93CF937E
:100D40001F930F930E9450060F900F900F900F90DB
:100D50000F900F909FEF29EF80E09150204080404E
:100D6000E1F700C000002196C031D105F9F663E03B
:100D700082E00E946A0999278131910511F174F48A
:100D800087309105F1F024F404970297F0F419C02C
:100D900089309105B1F00D97C1F413C08D319105E3
:100DA00081F034F48431910561F0499771F409C000
:100DB000843C910531F0873C910519F0813C910507
:100DC00021F481E080934C0102C010924C0163E059
:100DD00087E00E946A0991E0823009F090E09093E8
:100DE0004D01992341F08EE392E09F938F930E94EF
:100DF00050060F900F9023E042E063E082E00E94F3
:100E0000EA0981E392E09F938F930E9450060F902E
:100E10000F90C1E0D0E007E112E063E08C2F0E9468
:100E20006A09009771F09F938F93DF93CF931F937D
:100E30000F930E9450060F900F900F900F900F90FD
:100E40000F908FEF99EF20E0815090402040E1F724
:100E500000C000002196C031D105F9F6E7E3F1E0CA
:100E600080E18E0F11928E13FDCF0E94C5110E945A
:100E70000D098091BE0181608093BE0187E092E000
:100E80000E94B705569A5E98DF91CF911F910F91FE
:100E90000895CF93DF938FE79BEB0197F1F700C0A5
:100EA00000000E94E609EC01009711F481E0C3C044
:100EB00097FD05C080914701816080934701D7FF6E
:100EC00005C0809147018E7F809347012D2F3327E6
:100ED0002F733327BE016F737727C6FF02C060549C
:100EE0007109D6FF02C02054310940913601042E09
:100EF000000C550B649FC001659F900D749F900D71
:100F0000112481386FEF960714F481E89FEF9195D3
:100F10008195910981386FEF960714F481E89FEF6E
:100F2000819580934801249FC001259F900D349F97
:100F3000900D112481382FEF920714F481E89FEF70
:100F400091958195910981386FEF960714F481E8A6
:100F50009FEF8195809349018091BE0183FF60C01E
:100F600081EF91E00E94B705DF93CF938BEE91E084
:100F70009F938F930E94500689EE91E00E94B705DF
:100F800088ED91E00E94B70580913601282F082E48
:100F9000000C330B3F938F9383ED91E09F938F93DE
:100FA0000E94500681ED91E00E94B70580914701B3
:100FB0001F928F938CEC91E09F938F930E94500629
:100FC0008AEC91E00E94B70580914801282F082EF5
:100FD000000C330B3F938F9387EC91E09F938F939B
:100FE0000E94500685EC91E00E94B705809149016E
:100FF000282F082E000C330B3F938F9382EC91E047
:101000009F938F930E9450068FEB91E00E94B7054B
:101010008DB79EB744960FB6F8949EBF0FBE8DBF96
:1010200087E491E00E941A128091360191E08830A5
:101030000CF090E0890F80933601DF91CF910895F5
:101040001F93CF93DF93C0910001D09101018FEFE7
:101050009FEF9093010180930001CF3F8FEFD8075E
:1010600009F06AC08FE79BEB0197F1F700C0000021
:1010700082E00E94E309EC01892B09F05DC08091B8
:101080004D01882309F458C087E00E94E3090097C6
:1010900009F452C09C012F77332722303105A1F08B
:1010A00048F42115310569F02130310599F4807833
:1010B0008A641AC02330310551F02F373105A1F071
:1010C00009C08078826410C0807889640DC08078FF
:1010D00088640AC08CEA91E09F938F930E94500627
:1010E0000F900F9081E18FC0292F33272F7733275F
:1010F0002130310579F050F02230310579F023307C
:10110000310581F4EC01D078D86416C0EC01D078B8
:10111000D26412C0EC01D078DA640EC0EC01D07851
:10112000D9640AC089E991E09F938F930E94500689
:101130000F900F9080E167C08091BE0181FF18C0C1
:10114000209709F45DC085E891E00E94B705DF9320
:10115000CF9380E891E09F938F930E9450068EE793
:1011600091E00E94B7050F900F900F900F9003C071
:10117000209709F445C0CF379FE7D90711F48FE7CF
:1011800005C0CF3F8FEFD80721F48FEF0E9459069B
:1011900039C02D2F3327822F1C2F2F3F310581F48B
:1011A000DF93CF9380E691E09F938F930E94500648
:1011B0000E9479060F900F900F900F908C2F23C0F4
:1011C00090914C01992381F0A9014F775527423323
:1011D000510521F42078822F8A6006C04A305105DB
:1011E00019F42078822F82630E9459061F3F51F024
:1011F000DC2FCC27CF6FD0930101C093000102C038
:1012000080E001C081E0DF91CF911F910895E82F28
:10121000F0E0E95CFE4F80810895682F609582E0E0
:101220000C94240A509A83E091E00197F1F700C0F2
:10123000000050989AEB9A95F1F700C00895509AE3
:101240008AEB8A95F1F700C0509883E091E001970E
:10125000F1F700C000000895EF92FF920F931F93E3
:10126000CF93DF93C0E0D0E090E8E92EF12C082F77
:1012700010E0C7010C2E02C0959587950A94E2F7FD
:1012800080239123892B19F00E941F0902C00E941C
:1012900012092196C830D10561F7DF91CF911F91D6
:1012A0000F91FF90EF900895489B06C023E02A9588
:1012B000F1F700000197C1F70895489906C023E0AF
:1012C0002A95F1F700000197C1F7089558985098B2
:1012D00008950895CF92DF92EF92FF920F931F939C
:1012E000CF93DF931F92CDB7DEB7182FF894509AA3
:1012F00083EF9BE00197F1F700C0000069830E9433
:101300001F0969816C6020E1129FC0011124862BA6
:101310000E942C090E94120984EF91E00E945D094D
:10132000892B21F4789482EE9FEF43C084EF91E003
:101330000E945409009711F478943BC011E1C12C2C
:10134000D12C02E882E890E00E945D097C018823AC
:1013500051F199270E945409882329F1CC0CDD1CF6
:10136000902F9E19E81A9E1518F46894C0F806C0CC
:10137000113121F478948CEE9FEF1BC0115011F7BE
:101380008FE591E00E945D09892B21F478948BEE22
:101390009FEF0FC08BE590E00E945409892BB1F7B5
:1013A0007894C60106C07894812F90E0919581953C
:1013B00091090F90DF91CF911F910F91FF90EF90C6
:1013C000DF90CF90089560E00C946A0960E083E0BC
:1013D0000C946A091F93CF93DF9300D01F92CDB76F
:1013E000DEB7182FF894509A83EF9BE00197F1F73E
:1013F00000C000002B834A8369830E941F09698112
:10140000686030E1139FC0011124862B0E942C09D3
:101410000E9412098FE193E00197F1F700C00000EC
:101420000E941F094A81842F0E942C092B81822F40
:101430000E942C090E94120978940F900F900F902F
:10144000DF91CF911F910895262F277040E062E031
:101450000C94EA0980915A0108959FB7F89410926C
:1014600051019FBF9091D301943009F057C09091E2
:10147000E9009F703091EC00232F217030FD20E8AF
:10148000922B24E02093E9002091EB0020FF43C041
:101490002091EE0027FF3FC020914E01222321F032
:1014A0002091E80025FF37C010924E0126E03091D0
:1014B000E80035FD15C03091D301343061F530912D
:1014C000EB0035FD28C0215021F481E080934E01CE
:1014D00022C0EFE9FFE03197F1F700C00000E7CF4D
:1014E0008093F1008091E80085FD0AC08091E800BA
:1014F00080FFFCCF8091E8008E778093E80006C0E3
:101500008FB7F89421E0209351018FBF9F70909383
:10151000E90080E008959F709093E9008FEF0895AF
:10152000CF93DF9300D01F92CDB7DEB79C0180919F
:10153000D301843019F593E099833B832A839093F8
:10154000E9008FEF9091E800815095FD06C095ED80
:101550009A95F1F700008111F5CF8091E80085FFA1
:101560000DC040E050E063E070E0CE0101960E94C3
:10157000490D8091E8008E778093E8000F900F90DE
:101580000F90DF91CF910895CF93DF9300D01F92FA
:10159000CDB7DEB72091D301243021F522E0298395
:1015A0009B838A8383E08093E9008FEF9091E8002A
:1015B000815095FD06C095ED9A95F1F700008111D7
:1015C000F5CF8091E80085FF0DC040E050E063E07A
:1015D00070E0CE0101960E94490D8091E8008E775F
:1015E0008093E8000F900F900F90DF91CF910895B6
:1015F0002091D3012430F1F422E02093E9002FEF71
:101600003091E800215035FD06C035ED3A95F1F7EF
:1016100000002111F5CF2091E80025FF0BC040E02C
:1016200050E065E070E00E94490D8091E8008E77FF
:101630008093E8000895CF93DF932091D301243065
:1016400039F521E02093E9002FEF3091E800215097
:1016500035FD06C035ED3A95F1F700002111F5CFC3
:101660002091E80025FF14C0EC0140E050E068E064
:1016700070E00E94490D8091E8008E778093E80029
:1016800088E0FE01A2E5B1E001900D928A95E1F7B4
:10169000DF91CF91089587EA92E00E94B70580918B
:1016A000D201811109C00E94DE0E0E943B0F809181
:1016B000E20084608093E200089583EA92E00E9451
:1016C000B7051092D2010895089520914F012F5F20
:1016D000822F62E30E943027992319F020934F0153
:1016E000089510924F0180915101882371F18091EA
:1016F000D301843041F58091E9008F702091EC0096
:10170000922F917020FD90E8892B94E09093E9004E
:101710009091EB0090FF14C09091EE0097FF10C0E5
:101720009091E80095FF03C01092F100F9CF9091DD
:10173000E80090FF05C09091E8009E779093E80044
:101740008F708093E90010925101089542E061EC9E
:1017500081E00E94580E42E061EC82E00E94580E47
:1017600042E061EC83E00E94580E42E261EC84E0CA
:101770000C94580E8091D501833009F453C030F495
:10178000813071F0823009F48CC008958A3009F4F8
:1017900078C08B3009F45EC0893009F09AC020C04F
:1017A0008091D401813A09F094C08091E800877F4C
:1017B0008093E8008091D8019091D901892B21F480
:1017C00068E082E591E003C060E080E090E070E0D6
:1017D0000E94940D8091E8008B778093E800089533
:1017E0008091D401813209F074C08091D801909128
:1017F000D901892B09F06DC08091E800877F809323
:10180000E8008091E80082FD05C08091D30181113C
:10181000F8CF5FC08091F10080935A018091E80079
:101820008B7753C08091D401813A09F052C08091E6
:10183000D8019091D901892B09F04BC08091E80023
:10184000877F8093E8008091E80080FFFCCF809143
:101850000C0136C08091D4018132D9F58091D80134
:101860009091D901892BA9F58091E800877F809319
:10187000E8000E948D0E8091D60180930C010C949B
:101880004A188091D401813221F58091E800877F48
:101890008093E8000E948D0E8091D70180935B01B8
:1018A00008958091D401813AA1F48091E800877F66
:1018B0008093E8008091E80080FFFCCF80915B017D
:1018C0008093F1008091E8008E778093E8000C947B
:1018D0008D0E08950895089580915A0180935001C6
:1018E00010925A0180E00E940D090E944A130C9444
:1018F0004A180C946C0C0E944E1E8091D1018823D2
:1019000029F00E94771E81110C94330D089584B73D
:10191000877F84BF0FB6F894A89580916000886196
:1019200080936000109260000FBE90E080E80FB6D8
:10193000F89480936100909361000FBE8DE29AE06D
:101940000E941F1E8BE992E00E94B7050E946A0C5C
:101950000E9481120E94DE0E0E943B0F8091E200E5
:1019600084608093E20078948091D3018430E1F721
:101970008AE892E00E94B7050E94831282E091E01B
:101980000E94C01189E792E00E94B7050E946B0C8B
:101990008091D301853019F40E947B0CF9CF0E940D
:1019A0008912F6CF0E948B1E8091500180935A01BC
:1019B00008950C94D20C292F332723303105C9F018
:1019C00064F42130310581F02230310509F043C043
:1019D00084E790E02FEE32E042C021323105F1F091
:1019E0002232310541F137C082E190E023E633E055
:1019F00036C099278130910541F08230910541F040
:101A0000892B49F5EBEEF2E005C0EBEDF2E002C008
:101A1000EBEAF2E0849190E09F0121C06430D8F4B9
:101A2000E62FF0E0EE0FFF1FEF5DFE4F20813181CA
:101A300089E090E014C0643070F470E0FB01EE0FB8
:101A4000FF1FE75EFE4F20813181FB01EB5EFE4F01
:101A5000808190E004C080E090E020E030E0FA0176
:101A600031832083089580E189BD82E189BD09B475
:101A700000FEFDCF8091D8008F7D8093D8008091AB
:101A8000E00082608093E0008091E00081FDFCCF67
:101A90000895CF92DF92EF92FF920F931F93CF930F
:101AA000DF93EC018B016A010E94AC0E811133C0FF
:101AB000C114D10439F0F60180819181081B190B02
:101AC000C80FD91FE12CF12C0115110519F18091D6
:101AD000E80085FD16C08091E8008E778093E800CD
:101AE000C114D10449F0F60180819181E80EF91EFC
:101AF000F182E08285E00FC00E94AC0E882321F3C2
:101B00000AC089918093F10001501109FFEFEF1A8B
:101B1000FF0ADACF80E0DF91CF911F910F91FF9004
:101B2000EF90DF90CF9008952091DA013091DB01A2
:101B30002617370748F06115710539F42091E80040
:101B40002E772093E80001C0B90140E061157105CE
:101B5000A9F12091D301222309F443C0253009F4CF
:101B600042C02091E80023FD40C02091E80022FD02
:101B700032C02091E80020FFE9CF4091F30020918E
:101B8000F20030E0342BFC01CF016115710559F0F2
:101B90002830310540F481918093F1006150710942
:101BA0002F5F3F4FF1CF41E02830310509F040E091
:101BB0002091E8002E772093E800C8CF4111C9CFCB
:101BC0000AC08091D301882361F0853061F0809153
:101BD000E80083FD0AC08091E80082FFF2CF80E038
:101BE000089582E0089583E0089581E008952091AA
:101BF000DA013091DB012617370748F061157105CE
:101C000039F42091E8002E772093E80001C0B90153
:101C1000FC0120E06115710591F18091D3018823C9
:101C200009F440C0853009F43FC08091E80083FD8D
:101C30003DC08091E80082FD2FC08091E80080FFC8
:101C4000E9CF2091F3008091F20090E0922B611592
:101C5000710559F08830910540F424912093F100EA
:101C60003196615071090196F2CF21E0089709F091
:101C700020E08091E8008E778093E800CBCF21119F
:101C8000CCCF0AC08091D301882361F0853061F008
:101C90008091E80083FD0AC08091E80082FFF2CFC6
:101CA00080E0089582E0089583E0089581E008953A
:101CB000982F973058F59093E900981739F0709164
:101CC000EC002091ED005091F00003C0242F762FFE
:101CD00050E021FF19C03091EB003E7F3093EB00C4
:101CE0003091ED003D7F3093ED003091EB0031609D
:101CF0003093EB007093EC002093ED005093F000D4
:101D00002091EE0027FF07C09F5FD3CF8F70809395
:101D1000E90081E0089580E008958091D40187FF73
:101D200011C08091E80082FD05C08091D30181112E
:101D3000F8CF11C08091E8008B770BC08091D30160
:101D4000882349F08091E80080FFF8CF8091E80077
:101D50008E778093E80008952091E4003091E500AB
:101D600095E64091EC00842F817040FF22C0809165
:101D7000E80080FD1CC08091D301882391F085305C
:101D800091F08091EB0085FD10C04091E4005091EE
:101D9000E5004217530729F39A01915011F784E0A7
:101DA000089582E0089583E0089581E0089580E039
:101DB00008954091E80042FFDECF08950E944C0F45
:101DC0000E94540FE0EEF0E0808181608083E8EDB6
:101DD000F0E080818F77808319BCA7EDB0E08C9113
:101DE0008E7F8C9380818F7E80831092D2010895A4
:101DF0000F931F93CF93DF930E944C0F0E94540FB9
:101E0000C8EDD0E088818F77888388818068888357
:101E100088818F7D888319BC1092D3011092CF01E5
:101E20001092D1011092D00100EE10E0F8018081F3
:101E30008B7F808388818160888342E060E080E0DE
:101E40000E94580EE1EEF0E080818E7F8083E2EE0A
:101E5000F0E0808181608083808188608083F801E8
:101E600080818E7F8083888180618883DF91CF919C
:101E70001F910F910895E8EDF0E080818F7E8083BF
:101E8000E7EDF0E080818160808384E082BF81E0C3
:101E90008093D2010C94F80EE8EDF0E080818E7F03
:101EA00080831092E20008951092DA001092E1000F
:101EB00008951F920F920FB60F9211242F933F9304
:101EC0004F935F936F937F938F939F93AF93BF9342
:101ED000EF93FF938091E10082FF0BC08091E200BD
:101EE00082FF07C08091E1008B7F8093E1000E9418
:101EF000650B8091DA0080FF1FC08091D80080FFC1
:101F00001BC08091DA008E7F8093DA008091D90027
:101F100080FF0DC080E189BD82E189BD09B400FE6A
:101F2000FDCF81E08093D3010E944B0B05C019BC0B
:101F30001092D3010E945D0B8091E10080FF19C0D7
:101F40008091E20080FF15C08091E2008E7F809337
:101F5000E2008091E20080618093E2008091D800ED
:101F600080628093D80019BC85E08093D3010E94E1
:101F7000790C8091E10084FF30C08091E20084FF01
:101F80002CC080E189BD82E189BD09B400FEFDCF8E
:101F90008091D8008F7D8093D8008091E1008F7E62
:101FA0008093E1008091E2008F7E8093E200809137
:101FB000E20081608093E2008091CF01882311F0DC
:101FC00084E007C08091E30087FD02C081E001C08A
:101FD00083E08093D3010E94D90C8091E10083FFBC
:101FE00029C08091E20083FF25C08091E100877FB6
:101FF0008093E10082E08093D3011092CF01809121
:10200000E1008E7F8093E1008091E2008E7F8093DB
:10201000E2008091E20080618093E20042E060E0B3
:1020200080E00E94580E8091F00088608093F0005C
:102030000E94640BFF91EF91BF91AF919F918F919F
:102040007F916F915F914F913F912F910F900FBEB4
:102050000F901F9018951F920F920FB60F92112498
:102060002F933F934F935F936F937F938F939F93A0
:10207000AF93BF93CF93DF93EF93FF93C091E900AA
:10208000CF708091EC00D82FD17080FDD0E81092F5
:10209000E9008091F000877F8093F00078940E949F
:1020A0006F101092E9008091F00088608093F0003A
:1020B000CD2BCF70C093E900FF91EF91DF91CF91CD
:1020C000BF91AF919F918F917F916F915F914F9150
:1020D0003F912F910F900FBE0F901F9018951F9357
:1020E000CF93DF93CDB7DEB7AA970FB6F894DEBFD4
:1020F0000FBECDBFE4EDF1E088E08E0F9091F100CE
:1021000091938E13FBCF0E94BA0B8091E80083FF5E
:102110001FC18091D4019091D501492F50E04A30E0
:10212000510508F015C1FA01EA5AFF4F0C945027E7
:10213000803881F0823809F00BC18091D8018F700E
:102140008093E9008091EB0085FB882780F910924D
:10215000E90006C08091D0019091D1019111826077
:102160009091E800977F9093E8008093F10010929F
:10217000F100C8C0282F2D7F09F0EAC0882319F08C
:10218000823061F0E5C08091D601813009F0E0C075
:10219000933009F080E08093D1012BC08091D6016B
:1021A000811127C08091D8018F7009F4D1C080932C
:1021B000E9002091EB0020FF1CC0933021F48091B6
:1021C000EB00806214C09091EB0090619093EB0063
:1021D00021E030E0A90102C0440F551F8A95E2F7C3
:1021E0004093EA001092EA008091EB0088608093AF
:1021F000EB001092E9008091E800877F86C0811192
:10220000A7C01091D6011F778091E3008078812BC1
:102210008093E3008091E800877F8093E8000E942C
:102220008D0E8091E80080FFFCCF8091E3008068F4
:102230008093E300111102C082E001C083E080932B
:10224000D30186C08058823008F082C08091D601C8
:102250009091D7018C3D53E0950779F583E08A830F
:102260008AE289834FB7F894DE01139620E03EE0BE
:1022700051E2E32FF0E050935700E49120FF03C0B8
:10228000E295EF703F5FEF708E2F90E0EA3010F034
:10229000C79601C0C0968D939D932F5F243149F757
:1022A0004FBF8091E800877F8093E8006AE270E08A
:1022B000CE0101960E94940D14C0AE014F5F5F4F96
:1022C0006091D8010E94DB0CBC01892B09F440C04D
:1022D0009091E800977F9093E80089819A810E940D
:1022E000F70D8091E8008B778093E80031C080384B
:1022F00079F58091E800877F8093E8008091CF0195
:102300008093F1008091E8008E778093E8000E942E
:102310008D0E1EC081111CC09091D6019230C0F468
:102320008091E800877F8093E8009093CF010E941E
:102330008D0E8091CF01811106C08091E30087FD51
:1023400002C081E001C084E08093D3010E94A60B0B
:102350008091E80083FF0AC08091E800877F809326
:10236000E8008091EB0080628093EB00AA960FB6A4
:10237000F894DEBF0FBECDBFDF91CF911F910895BE
:1023800090936101809360010895E0916001F09164
:102390006101309721F00190F081E02D099480E0F7
:1023A0000895EF92FF920F931F93CF93DF93E091E5
:1023B0006001F09161013097B1F18C010280F381ED
:1023C000E02D09958091BE0182FF2DC080FF04C0E1
:1023D00080E894E00E94B705E80118E08AE7E82E5B
:1023E00084E0F82E8091BE0180FF0BC088811F928F
:1023F0008F93FF92EF920E9450060F900F900F90D4
:102400000F90115021961111EDCF8091BE0180FFE8
:102410000AC088E794E0DF91CF911F910F91FF9060
:10242000EF900C94B705DF91CF911F910F91FF9022
:10243000EF900895E0916001F0916101309721F0F3
:102440000480F581E02D09940895CF93DF93EC018A
:1024500080915E0190915F01C817D90709F1D0936F
:102460005F01C0935E01E0916001F09161013097DE
:10247000B9F00680F781E02DCE0109958091BE016B
:1024800082FF0EC080FF0CC0DF93CF938AE694E0FA
:102490009F938F930E9450060F900F900F900F9074
:1024A000DF91CF910895CF93DF93EC0180915C0190
:1024B00090915D01C817D90709F1D0935D01C093D0
:1024C0005C01E0916001F09161013097B9F0008406
:1024D000F185E02DCE0109958091BE0182FF0EC0ED
:1024E00080FF0CC0DF93CF938AE594E09F938F9396
:1024F0000E9450060F900F900F900F90DF91CF9198
:1025000008950C944B130E94B81E0E9479060C94F7
:102510006909CF92DF92EF92FF920F931F93CF93AF
:10252000DF9300D000D000D0CDB7DEB70E942008E6
:1025300083E6C82E81E0D82E00E010E0E02E802F48
:102540000E940709F60141916F01F42EF826B1F4BB
:102550000F5F1F4F0031110589F78FEF89838A8341
:102560001B820E94C11E8160782F9D838C834981CC
:102570005A816B818D810E949D1347C09091BE014D
:1025800091FF04C08E830E9467138E8120E030E0AB
:102590004F2D50E0922FBA01022E02C0759567951B
:1025A0000A94E2F760FF2BC02983EA8221E030E041
:1025B000690102C0CC0CDD1C9A95E2F790E08C21F9
:1025C0009D21892B09F420E02B830E94C11E81608C
:1025D000782F9D838C8349815A816B818D810E94E4
:1025E0009D1349815A816B817C818D810E943B1EA4
:1025F000F801ED59FE4F8081C826C08206C02F5FCA
:102600003F4F2830310531F6A3CF0E943A1E0E9479
:1026100082210E944907109162010E94C51118177A
:1026200041F10E94C511809362019091BE0192FF19
:102630000EC090FF0CC01F928F938BE894E09F9385
:102640008F930E9450060F900F900F900F908091E3
:10265000620126960FB6F894DEBF0FBECDBFDF91A4
:10266000CF911F910F91FF90EF90DF90CF900C943E
:102670004C1E26960FB6F894DEBF0FBECDBFDF917D
:10268000CF911F910F91FF90EF90DF90CF90089521
:102690000C940D0908950895CF93DF931F92CDB741
:1026A000DEB769830E94070990E021E030E069818C
:1026B00002C0220F331F6A95E2F72823392381E0F5
:1026C000232B09F480E00F90DF91CF910895EF92D2
:1026D000FF920F931F93CF93DF9384EA94E00E94BD
:1026E000B705C0E0D0E089E2E82E81E0F82E06E9E7
:1026F00014E08C2F0E9407090E94241EFF92EF9283
:102700001F928F93DF93CF931F930F930E945006D6
:1027100021968DB79EB708960FB6F8949EBF0FBE50
:102720008DBFC031D10529F7DF91CF911F910F9156
:10273000FF90EF90089508950895CF93DF93CDB75C
:10274000DEB72B970FB6F894DEBF0FBECDBF942F28
:102750004F83252F588769877A878B874A855B85C2
:10276000452B21F02F3F09F59F3FF9F4DE0111962B
:1027700086E0FD0111928A95E9F785E0FE01379622
:1027800001900D928A95E1F749815A816B817C8194
:102790008D819E810E94F51A2B960FB6F894DEBFAC
:1027A0000FBECDBFDF91CF9108954F8158856985C8
:1027B0007A858B850E943B1ED9CFCF93882309F45D
:1027C000A9C0C82F8238A1F40E94C51181FDA2C002
:1027D00089E30E94801D0E94F91D2FEF81EE94E095
:1027E000215080409040E1F700C0000089E315C00F
:1027F0008338C1F40E94C51180FD8CC083E50E941E
:10280000801D0E94F91D2FEF81EE94E02150804041
:102810009040E1F700C0000083E50E949D1DCF912C
:102820000C94F91D8438A1F40E94C51182FD72C078
:1028300087E40E94801D0E94F91D2FEF81EE94E035
:10284000215080409040E1F700C0000087E4E5CFD0
:102850008CEF8C0F813A20F080E58C0F8E3248F49B
:102860008C2F0E94AC24811155C08C2F0E94801D9A
:10287000D6CF80E28C0F883048F4C77081E001C069
:10288000880FCA95EAF70E94BF1DC9CF8BE58C0F50
:10289000833078F4C53A29F0C63A31F083E890E005
:1028A00005C081E890E002C082E890E0CF910C94EE
:1028B000251288E58C0F853168F5C83A89F0C93A48
:1028C00091F0CA3A99F0CB3AA1F0CC3AA9F0CD3ABE
:1028D000B1F0CE3AB9F0CF3AC1F080E090E017C045
:1028E00082EE90E014C089EE90E011C08AEE90E094
:1028F0000EC085EB90E00BC086EB90E008C083EB48
:1029000090E005C084EB90E002C087EB90E0CF91AF
:102910000C945312CF910895882309F46AC0823829
:10292000A1F40E94C51181FF64C089E30E94801D4B
:102930000E94F91D2FEF81EE94E0215080409040DD
:10294000E1F700C0000089E315C08338B9F40E94A4
:10295000C51180FF4EC083E50E94801D0E94F91DB5
:102960002FEF81EE94E0215080409040E1F700C0CD
:10297000000083E50E949D1D0C94F91D8438A1F48C
:102980000E94C51182FF35C087E40E94801D0E940D
:10299000F91D2FEF81EE94E0215080409040E1F747
:1029A00000C0000087E4E6CF9CEF980F913A10F347
:1029B00090E5980F9E32F0F290E2980F983050F424
:1029C000877091E001C0990F8A95EAF7892F0E94DC
:1029D000C51DD2CF9BE5980F933020F480E090E0A6
:1029E0000C942512885A853120F480E090E00C94F4
:1029F00053120895882321F00E94BF1D0C94F91DE5
:102A00000895882321F00E94C51D0C94F91D089596
:102A1000BF92CF92DF92EF92FF920F931F93CF93CB
:102A2000DF9300D000D000D0CDB7DEB725E0FC01A9
:102A3000DE01119601900D922A95E1F7FC0140818B
:102A40003181F280258122952F7063817481672BFB
:102A500009F4FEC23F3F19F44F3F09F4F9C26C017B
:102A600049833A8389819A812E830E943F1D182FC2
:102A7000B92E0E943E1D0E944E1CEB2DE295EF7078
:102A8000F0E0E05AFF4F2E810C9450278B2D807F71
:102A90009B2D9F70092F882311F00295007FFF2046
:102AA00049F0002309F481C2802F0E94D21D0E94A8
:102AB000F91D7BC2812F0E948C14002309F4C8C227
:102AC000802F0E94D81D26960FB6F894DEBF0FBE49
:102AD000CDBFDF91CF911F910F91FF90EF90DF90CD
:102AE000CF90BF900C94F91D8B2D807F9B2D9F70F4
:102AF000092F803211F00295007F112319F0113057
:102B000009F12AC0FF20B1F0802F222351F121309A
:102B100041F526960FB6F894DEBF0FBECDBFDF910C
:102B2000CF911F910F91FF90EF90DF90CF90BF90CA
:102B30000C94E21D222319F0213009F489C20E946D
:102B4000E51D2DC0FF20F1F0263008F081C20E9463
:102B5000BC1D802329F023C0FF20F9F0211116C0ED
:102B6000802F26960FB6F894DEBF0FBECDBFDF9143
:102B7000CF911F910F91FF90EF90DF90CF90BF907A
:102B80000C94FA14253008F063C209C0F60185815F
:102B900080FF0BC28F708583E3CF21111BC2802F72
:102BA00082C12B2D26952695237030E02115310505
:102BB00021F021303105D1F04BC2FF2021F0812FCF
:102BC0009B2D937002C080E090E026960FB6F8949B
:102BD000DEBF0FBECDBFDF91CF911F910F91FF9050
:102BE000EF90DF90CF90BF900C942512FF2021F042
:102BF000812F9B2D937002C080E090E026960FB647
:102C0000F894DEBF0FBECDBFDF91CF911F910F9122
:102C1000FF90EF90DF90CF90BF900C945312812FD4
:102C2000FF2019F00E94082002C00E947020269602
:102C30000FB6F894DEBF0FBECDBFDF91CF911F91CD
:102C40000F91FF90EF90DF90CF90BF900C94F52004
:102C50008B2D837009F07BC0F110FAC1812F829512
:102C600086958770880F880F912F9F70C92ED12C61
:102C7000E12CF12C082E04C0CC0CDD1CEE1CFF1C3A
:102C80000A94D2F714FF12C04FE050E060E070E009
:102C900004C0440F551F661F771F8A95D2F7CB01DA
:102CA000BA01609570958095909503C060E070E0E2
:102CB000CB012B2D269526952370422F50E04230D4
:102CC0005105D9F04330510569F16C297D298E29D0
:102CD0009F294130510551F126960FB6F894DEBF79
:102CE0000FBECDBFDF91CF911F910F91FF90EF905D
:102CF000DF90CF90BF900C94631C6C297D298E29A6
:102D00009F2926960FB6F894DEBF0FBECDBFDF9188
:102D1000CF911F910F91FF90EF90DF90CF90BF90D8
:102D20000C94751C0E94631CC701B60126960FB651
:102D3000F894DEBF0FBECDBFDF91CF911F910F91F1
:102D4000FF90EF90DF90CF90BF900C94511CFF202C
:102D500019F08B2D817001C08695882309F478C104
:102D6000812F829586958770880F880F912F9F708D
:102D7000C92ED12CE12CF12C082E04C0CC0CDD1C6A
:102D8000EE1CFF1C0A94D2F714FF12C04FE050E073
:102D900060E070E004C0440F551F661F771F8A95DE
:102DA000D2F7CB01BA01609570958095909503C0DC
:102DB00060E070E0CB012B2D269526952370422FE5
:102DC00050E042305105D9F04330510569F16C298A
:102DD0007D298E299F294130510551F126960FB644
:102DE000F894DEBF0FBECDBFDF91CF911F910F9141
:102DF000FF90EF90DF90CF90BF900C941A1D6C293C
:102E00007D298E299F2926960FB6F894DEBF0FBE26
:102E1000CDBFDF91CF911F910F91FF90EF90DF9089
:102E2000CF90BF900C942C1D0E941A1DC701B601B3
:102E300026960FB6F894DEBF0FBECDBFDF91CF91BF
:102E40001F910F91FF90EF90DF90CF90BF900C9467
:102E5000081D103FC9F128F480E4810F803250F042
:102E60009FC0123F09F461C008F44AC0133F09F43F
:102E700071C096C0012F00718B2D8F71FF2051F012
:102E80000E94A11C812F002319F08295807F69CEBA
:102E90008F7067CE0E94C21C812F002319F082958B
:102EA000807F01C08F7026960FB6F894DEBF0FBEEC
:102EB000CDBFDF91CF911F910F91FF90EF90DF90E9
:102EC000CF90BF900C940115FF20B1F0253008F091
:102ED000BFC08B2D8F7126960FB6F894DEBF0FBE44
:102EE000CDBFDF91CF911F910F91FF90EF90DF90B9
:102EF000CF90BF900C94E71C263008F0A9C0E9CF12
:102F0000FF20A9F08B2D8F7126960FB6F894DEBFA7
:102F10000FBECDBFDF91CF911F910F91FF90EF902A
:102F2000DF90CF90BF900C94A11CFF2059F38B2D04
:102F30008F7126960FB6F894DEBF0FBECDBFDF911E
:102F4000CF911F910F91FF90EF90DF90CF90BF90A6
:102F50000C94C21CFF2099F08B2D8F7126960FB612
:102F6000F894DEBF0FBECDBFDF91CF911F910F91BF
:102F7000FF90EF90DF90CF90BF900C948C1C269622
:102F80000FB6F894DEBF0FBECDBFDF91CF911F917A
:102F90000F91FF90EF90DF90CF90BF900C94871C23
:102FA000FF20A9F0222309F4ADCF812F26960FB67A
:102FB000F894DEBF0FBECDBFDF91CF911F910F916F
:102FC000FF90EF90DF90CF90BF900C94DD13222301
:102FD00009F4ADCF812F26960FB6F894DEBF0FBE51
:102FE000CDBFDF91CF911F910F91FF90EF90DF90B8
:102FF000CF90BF900C948C144B2D4F70612FC60155
:103000000E94821F26960FB6F894DEBF0FBECDBF7A
:10301000DF91CF911F910F91FF90EF90DF90CF90B4
:10302000BF900C94991B4B2D4F70612FC6012696B3
:103030000FB6F894DEBF0FBECDBFDF91CF911F91C9
:103040000F91FF90EF90DF90CF90BF900C94851F71
:1030500026960FB6F894DEBF0FBECDBFDF91CF919D
:103060001F910F91FF90EF90DF90CF90BF90089548
:103070000E94DF1D0E94AE1D0E94F91D0E942722A2
:103080000E94F52080E090E00E94251280E090E010
:103090000C9453120E94CF1D0C9438180E943F1DAF
:1030A000292F22952F7030E02C3031054CF42A3036
:1030B0003105C4F4225031092230310540F023C0DB
:1030C0002C303105D1F02F303105B9F01CC0853AD4
:1030D00028F48430B0F4823028F413C090E2980FC2
:1030E000983078F0883E30F4803E58F48450813A2D
:1030F00050F407C0803F39F404C093FB882780F95F
:10310000089581E0089580E00895CF93DF9300D083
:1031100000D01F92CDB7DEB70F900F900F900F9099
:103120000F90DF91CF910895CF93DF9300D000D01F
:1031300000D0CDB7DEB726960FB6F894DEBF0FBE2F
:10314000CDBFDF91CF9108951F93CF93DF93C091AF
:10315000730116E080917401C81799F0D0E01C9FAC
:10316000F0011D9FF00D1124EB58FE4F408151815D
:1031700062817381848195810E9494182196C77021
:10318000E9CFDF91CF911F9108954091A501509112
:10319000A6016091A7017091A8018091A901909169
:1031A000AA010C9494188091AA0182958F7009F05D
:1031B00054C08091A701882309F44FC08091730106
:1031C000A09174016091A5017091A6014091A801A0
:1031D0005091A901B6E08A1709F43FC090E041156B
:1031E0005105C1F17F3F11F46F3FA1F1B89FF0018C
:1031F000B99FF00D1124EB58FE4F218172132AC0A4
:103200002081621327C02281211124C023813481AF
:103210002417350710F421503109241B350B283CA5
:103220003105C0F42091AA012F7020612093AA01DA
:1032300026E0289FF001299FF00D1124E658FE4F4B
:1032400080818F708061808385EA91E00E940815FB
:103250000C94A41801968770BECF0895CF92DF9288
:10326000EF92FF920F931F93CF93DF93CDB7DEB70B
:1032700062970FB6F894DEBF0FBECDBF8C0185E01C
:10328000F801DE011D9601900D928A95E1F7D801B3
:103290004C9111965C91119712966C91129713961E
:1032A000CD90DC9014973091A5017091A60180918A
:1032B000A8019091A901009709F46BC17F3F19F40F
:1032C0003F3F09F466C1E090A701EE2009F4C0C0B9
:1032D0002091AA01C816D90628F0F601E81BF90BBF
:1032E000CF0104C0809590958C0D9D1DFF24F39413
:1032F000883C910578F0F12C207F09F0C6C07C2D28
:10330000D98AC88A89890E94851885EA91E00E9435
:103310000815B1C0822F807F09F046C0751314C014
:10332000341312C0611110C02F7020612093AA01C4
:103330000E94C51885EA91E00E9408158091AA01B3
:10334000D80115968C932EC0CD2819F15F3F11F44A
:103350004F3FF9F0F62E61111CC08091730120914E
:10336000740136E0821709F45AC090E0389FF001EA
:10337000399FF00D1124EB58FE4F7181571306C091
:103380007081471303C07281711103C00196877069
:10339000E9CFF62E662309F418C18091AA01816055
:1033A0008093AA01F12C11C1751308C0341306C013
:1033B000611104C08091AA01D801C3C04D875E8706
:1033C0008D859E856A8B0E944E186A898823E1F15B
:1033D0006623D1F12091AA01822F82958F7090E00F
:1033E000029774F08091A5019091A60198878F8330
:1033F0001986DB86CA862C87CE0107960E9408159F
:1034000086E0F801A5EAB1E001900D928A95E1F716
:103410000E94D3180E94C518FF24F394D6C04D878C
:103420005E878D859E850E943F1D292F22952F70D6
:1034300030E0223031050CF0BCC09F7009F0B6C0FE
:10344000805E883008F4C1C0C8010E940815E4CF2E
:10345000C816D90608F453C0F601E81BF90BCF01D2
:10346000883C910508F450C0F12C7C2DD98AC88A7B
:1034700089890E948518E5EAF1E086E0DF011D9266
:103480008A95E9F70E94C518A0C0751314C03413BB
:1034900012C0611110C08091AA01F8018583C80192
:1034A0000E94081586E0E5EAF1E0DF011D928A95A9
:1034B000E9F7FE2C8AC04D875E878D859E856A8BD5
:1034C0000E944E186A89882309F4BECF662309F446
:1034D000BBCF2091AA01822F82958F7090E0029736
:1034E0000CF48ECF8091A5019091A6019A838983D7
:1034F0001B82DD82CC822E83CE0101967FCF809508
:1035000090958C0D9D1DACCFF62E662309F49CCFB3
:1035100075132EC034132CC02091AA0120FD1FC0AA
:10352000822F82958F70D9F0D80115962C9315971C
:103530008F3049F08F5F982F9295907F822F8F70F8
:10354000892B15968C93C8010E94081586E0F80116
:10355000A5EAB1E001900D928A95E1F793CF86E05C
:10356000F801A5EAB1E001900D928A95E1F72DC02E
:103570004D875E878D859E850E944E18811140CFB4
:103580008091AA0181608093AA01C8010E94081558
:103590001CC0662309F458CF4D875E878D859E85B4
:1035A0000E944E18882309F44FCF2ACF811148CFAB
:1035B0000CC0243031050CF047CF9F7009F440CF88
:1035C000F8019581907F09F03BCF8F2D62960FB661
:1035D000F894DEBF0FBECDBFDF91CF911F910F9149
:1035E000FF90EF90DF90CF9008951F93CF93DF93DC
:1035F000CDB7DEB72C970FB6F894DEBF0FBECDBFA8
:103600004F83588769877A878B879C87CE01079677
:103610000E942E19882369F08F8198852A853B8521
:10362000232BF1F19F3F09F063C08F3F09F060C089
:1036300037C086E0FE013796DE01119601900D92AB
:103640008A95E1F76F817885EA85FB85309741F1AE
:103650007F3F11F46F3F21F12091740130E0C901E7
:103660000196877099274091730150E08417950760
:1036700009F447C069837A83FD83EC8396E0929FC7
:10368000D001939FB00D1124AB58BE4FFE0131966F
:1036900001900D929A95E1F7809374010E94A4180D
:1036A00016E080917301909174018917C1F1189F00
:1036B000C00111248B589E4F0E942E19882379F146
:1036C000E09173011E9FF0011124EB58FE4F4081E1
:1036D000518162817381848195810E9494188091C7
:1036E000730190E001968770992780937301D9CF79
:1036F0004F81588569857A858B859C850E949418B1
:10370000CFCF0E944A181092740110927301E5EA1B
:10371000F1E086E0DF011D928A95E9F7C1CF2C9692
:103720000FB6F894DEBF0FBECDBFDF91CF911F91D2
:103730000895DF92EF92FF920F931F93CF93DF9341
:10374000FC01892B09F48AC0E12CF12CDD24D394EF
:10375000EF0121968491853709F461C058F48437CC
:1037600008F04EC0843008F06AC08130D1F0823059
:1037700071F174C0883709F45DC050F4863709F4DC
:1037800055C0873709F06AC08E2D0E94CC1D54C0E9
:103790009CE7980F903708F061C08F770E948C14D7
:1037A00050C08F010E5F1F4FFE01849190E2980F71
:1037B000983050F48770FD2D01C0FF0F8A95EAF70D
:1037C0008F2F0E94D21D14C00E94DD1313C08F01E1
:1037D0000E5F1F4FFE01C49180E28C0F883060F4B1
:1037E000C7708D2D01C0880FCA95EAF70E94D81DB9
:1037F0000E94F91DE80125C08C2F0E948C14FACF7D
:103800009F012E5F3F4FFE01C491CC2369F08FE9E9
:103810009FE00197F1F700C00000C150F6CF9F0173
:103820002E5F3F4FFE01F490E9010BC00E94BC1DCA
:10383000E82E07C00E94CF1D0E94F91D02C00E9401
:10384000DD138F2D882341F0EFE9FFE03197F1F789
:1038500000C000008150F6CFFE017ACFDF91CF91FA
:103860001F910F91FF90EF90DF9008956093AF014B
:103870007093B0018093B1019093B2010E944A1EEF
:103880000C9438186093AB017093AC018093AD0138
:103890009093AE010E944B1E0C94381808950C941E
:1038A000361C0F931F930091AF011091B00120912E
:1038B000B1013091B201602B712B822B932B1F91A0
:1038C0000F910C94361C0F931F930091AF01109130
:1038D000B0012091B1013091B201602371238223A4
:1038E00093231F910F910C94361C0F931F930091FB
:1038F000AF011091B0012091B1013091B201602768
:103900007127822793271F910F910C94361C60E03A
:1039100070E0CB010C94421C0F931F9341E050E0E8
:1039200060E070E08A019B0104C0000F111F221F9C
:10393000331F8A95D2F7C901B8011F910F910C94DA
:10394000421C0F931F9341E050E060E070E004C020
:10395000440F551F661F771F8A95D2F78091AB01E0
:103960009091AC01A091AD01B091AE018A019B0193
:10397000082B192B2A2B3B2BC901B8011F910F9142
:103980000C94421C0F931F9341E050E060E070E004
:1039900004C0440F551F661F771F8A95D2F74095C4
:1039A0005095609570958091AB019091AC01A0917C
:1039B000AD01B091AE018A019B01082319232A238E
:1039C0003B23C901B8011F910F910C94421C0F9326
:1039D0001F9341E050E060E070E004C0440F551FC9
:1039E000661F771F8A95D2F78091AB019091AC0149
:1039F000A091AD01B091AE018A019B010827192762
:103A00002A273B27C901B8011F910F910C94421C32
:103A10000F931F930091AB011091AC012091AD0168
:103A20003091AE01602B712B822B932B1F910F9144
:103A30000C94421C0F931F930091AB011091AC01A9
:103A40002091AD013091AE01602371238223932335
:103A50001F910F910C94421C0F931F930091AB0187
:103A60001091AC012091AD013091AE01602771271A
:103A7000822793271F910F910C94421C0895CF9297
:103A8000DF92EF92FF920F931F93CF93DF938C01FE
:103A9000C090AF01D090B001E090B101F090B201C0
:103AA0004091AB015091AC016091AD017091AE01BC
:103AB000C42AD52AE62AF72ACFE1D0E0D701C601E9
:103AC0000C2E04C0B695A795979587950A94D2F7C2
:103AD00080FF07C0B8018C2F0E94581F81309105CC
:103AE00031F4219758F7B80180E00E94581FDF9108
:103AF000CF911F910F91FF90EF90DF90CF9008959D
:103B000020910D0130910E01F90132969FEF40E0B6
:103B10005191581789F09F3F19F4511101C0942F0A
:103B20004F5F4630A9F79F3F39F0F901E90FF11DCA
:103B300097FDFA9582830895089520910D013091A3
:103B40000E01F9013296285F3F4F9081981301C012
:103B500010823196E217F307C1F7089581E090E0F3
:103B6000E0910D01F0910E01E80FF91F108201960E
:103B700088309105A9F708958091BD01089590912D
:103B8000BD01892B8093BD01089580959091BD0161
:103B900089238093BD0108958093BD0108951092FB
:103BA000BD0108959091BC01892B8093BC010895BB
:103BB00080959091BC0189238093BC010895109257
:103BC000BC0108958093B30108951092B301089544
:103BD00080910D0190910E01FC0131969C01285FAE
:103BE0003F4F80E0919191118F5FE217F307D1F77A
:103BF0000895E0910D01F0910E018091BD01808347
:103C0000E0910D01F0910E0190818091BC01892B12
:103C100080838091B301882361F0E0910D01F091E0
:103C20000E019081892B80830E94E81D81111092E2
:103C3000B30180910D0190910E010C94D1119093DC
:103C400035018093340108958295982F9C7C392FFB
:103C500036953695282F237344E0249FC001112404
:103C6000932F982B292F2A7A2695892F8575880FCF
:103C7000822B08950895CF93DF9300D000D01F9238
:103C8000CDB7DEB70F900F900F900F900F90DF9190
:103C9000CF910895089508950C9448138091D3010D
:103CA000843021F11092BF0120E488E190E00FB64A
:103CB000F894A895809360000FBE2093600083B7AE
:103CC000817F846083BF83B7816083BF7894889548
:103CD00083B78E7F83BF0FB6F894A895809160005C
:103CE000886180936000109260000FBE0895CF93AA
:103CF0000E949B130E9420080E949C13C0E08C2FFE
:103D00000E940709811104C0CF5FC031C1F701C013
:103D100081E0CF9108950E944A130C944A181F9293
:103D20000F920FB60F9211248F939F93AF93BF936F
:103D30008091BF01811113C08091C0019091C10198
:103D4000A091C201B091C3014196A11DB11D809304
:103D5000C0019093C101A093C201B093C301BF9170
:103D6000AF919F918F910F900FBE0F901F9018955C
:103D700082E084BD93E095BD9AEF97BD80936E007D
:103D800008952FB7F8948091C0019091C101A0913E
:103D9000C201B091C3012FBF08952FB7F89460916D
:103DA000C0017091C1018091C2019091C3012FBFE8
:103DB0000895CF92DF92EF92FF920F931F932FB748
:103DC000F8944091C0015091C1016091C20170917D
:103DD000C3012FBF6A017B01EE24FF248C0120E088
:103DE00030E0C016D106E206F30610F44150510946
:103DF0009A01281B390BC9011F910F91FF90EF9079
:103E0000DF90CF9008951F920F920FB60F9211245A
:103E10008F939F93AF93BF938091C0019091C10105
:103E2000A091C201B091C3010196A11DB11D809363
:103E3000C0019093C101A093C201B093C301BF918F
:103E4000AF919F918F910F900FBE0F901F9018957B
:103E50000E94DE0EF8942FEF87EA91E62150804011
:103E60009040E1F700C0000087E090EBDC01809318
:103E7000DC019093DD01A093DE01B093DF019CE0B3
:103E800088E10FB6F894A895809360000FBE9093D8
:103E90006000FFCF28E0929FF0011124E80FF11D90
:103EA000E052FF4F9491892F8F7092959F700895E3
:103EB000CF93C82FCB010E944A1F282F30E080E10A
:103EC000989FA0011124422B532B4038510519F41F
:103ED00080E090E015C09770E92FF0E088E0C89F7F
:103EE000E00DF11D112484E0EE0FFF1F8A95E1F72C
:103EF000E20FF31FEE0FFF1FE050F84985919491F8
:103F0000CF91089580E090E0089508958091C601D2
:103F100080FF0BC06091120185E0689FB001112401
:103F200075956795759567952BC081FF09C0609160
:103F3000120185E0689FB00111247595679520C036
:103F400082FF07C06091120185E0689FB0011124D3
:103F500017C09091C7019923D1F060911101961774
:103F600088F72091120185E0289F90011124929FEB
:103F7000A001939F500D112470E0CA010E943C27BC
:103F80006038710540F46115710539F002C065E0D3
:103F900070E0862F08958FE7089581E0089580915D
:103FA000C60180FF08C06091100170E075956795AB
:103FB0007595679521C081FF06C06091100170E082
:103FC0007595679519C082FF04C06091100170E07B
:103FD00010C09091C7019923C1F060910F0196170D
:103FE000A0F780911001899FC001112470E00E9408
:103FF0003C276038710528F46115710521F0862F82
:1040000008958FE7089581E0089561E070E0F4CFAE
:10401000803F21F40E94861F819504C0813F29F4CE
:104020000E94861F8093CA010895823F21F40E9456
:10403000861F819504C0833F29F40E94861F8093C8
:10404000C9010895893F19F40E94CF1F05C08A3F16
:1040500031F40E94CF1F81958093CB0108958B3F4F
:1040600021F40E94CF1F819504C08C3F29F40E9447
:10407000CF1F8093CC010895843F21F48091C80123
:10408000816017C0853F21F48091C801826011C012
:10409000863F21F48091C80184600BC0873F21F4E2
:1040A0008091C801886005C0883F31F48091C801C3
:1040B00080618093C80108958D3F21F48091C601ED
:1040C00081600BC08E3F21F48091C601826005C0E3
:1040D0008F3F29F48091C60184608093C6010895C2
:1040E000803F39F48091CA0187FF6CC01092CA01E9
:1040F00069C0813F29F48091CA011816BCF362C0DF
:104100009091C901823F29F497FF5CC01092C901C8
:1041100059C0833F19F41916CCF354C0893F41F4B8
:104120008091CB0118160CF04DC01092CB014AC003
:104130008A3F29F48091CB0187FF44C0F6CF8B3FA3
:1041400039F48091CC0187FF3DC01092CC013AC078
:104150008C3F29F48091CC011816BCF333C0843F06
:1041600021F48091C8018E7F17C0853F21F4809192
:10417000C8018D7F11C0863F21F48091C8018B7FDB
:104180000BC0873F21F48091C801877F05C0883F1D
:1041900031F48091C8018F7E8093C80113C08D3F98
:1041A00021F48091C6018E7F0BC08E3F21F4809157
:1041B000C6018D7F05C08F3F29F48091C6018B7F9A
:1041C0008093C6018091C90181110EC08091CA01FE
:1041D00081110AC08091CB01811106C08091CC0170
:1041E000811102C01092C70108958091BE0183FF22
:1041F0007EC089ED94E00E94B7058091C8011F92AE
:104200008F9384ED94E09F938F930E94500682EDEC
:1042100094E00E94B7058091C901282F082E000C58
:10422000330B3F938F938FEC94E09F938F930E9477
:1042300050068DEC94E00E94B7058091CA01282FAA
:10424000082E000C330B3F938F938AEC94E09F93DE
:104250008F930E94500688EC94E00E94B7058091ED
:10426000CB01282F082E000C330B3F938F9385EC46
:1042700094E09F938F930E94500683EC94E00E94F9
:10428000B7058091CC01282F082E000C330B3F93EB
:104290008F9380EC94E09F938F930E9450068DEB58
:1042A00094E00E94B7058091C7011F928F938AEB1B
:1042B00094E09F938F930E94500688EB94E00E94B5
:1042C000B7058091C6011F928F9385EB94E09F9371
:1042D0008F930E94500682EB94E00E94B7058DB741
:1042E0009EB74C960FB6F8949EBF0FBE8DBF88EC5C
:1042F00091E00E941A120E94C11E9093C501809302
:10430000C40108951F93CF93DF938091C4019091CE
:10431000C5010E94D91EAC019091C701992321F0DB
:104320002091130130E006C0209114018AE0289FFB
:10433000900111244217530708F485C08091C901E8
:10434000C091CA01D091CB011091CC01811107C05D
:10435000C11175C0D11173C0111171C074C09F3FDC
:1043600019F09F5F9093C701181624F40E94861FCE
:104370008093C9018091C90187FF05C00E94861FF3
:1043800081958093C9011C1624F40E94861F809396
:10439000CA018091CA0187FF05C00E94861F8195CE
:1043A0008093CA016091C901662331F1C091CA01AD
:1043B000CC2311F1062E000C770B880B990B0E9471
:1043C000372623E333E343E35FE30E949B260E9407
:1043D000FF256093C9016C2FCC0F770B880B990BCD
:1043E0000E94372623E333E343E35FE30E949B26E7
:1043F0000E94FF256093CA011D1624F40E94CF1F5E
:104400008093CB018091CB0187FF05C00E94CF1F15
:1044100081958093CB01111624F40E94CF1F8093C5
:10442000CC018091CC0187FF05C00E94CF1F8195F0
:104430008093CC01DF91CF911F910C94F5209F3F89
:1044400009F08FCF97CFDF91CF911F910895E8ECBE
:10445000F1E085E0DF011D928A95E9F71092C7012E
:104460001092C60108958CEF96E00E94B7051F9246
:1044700081E08F931F9285E08F938EEA96E09F9361
:104480008F930E9450060F900F900F900F900F90F7
:104490000F9008958330E9F128F4813061F0823083
:1044A00009F10895853009F462C008F449C08630E6
:1044B00009F474C0089580911401262F30E0280F6C
:1044C000311D2F3F310524F4680F6093140103C0A0
:1044D0008FEF80931401809114011F928F9387EEC8
:1044E00095E072C080911301262F30E0280F311D16
:1044F0002F3F310524F4680F6093130103C08FEF41
:1045000080931301809113011F928F9385ED95E0A5
:104510005BC080911201262F30E0280F311D2F3F04
:10452000310524F4680F6093120103C08FEF80936C
:104530001201809112011F928F9382EC95E044C08A
:1045400080911101262F30E0280F311D2F3F3105BA
:1045500024F4680F6093110103C08FEF8093110161
:10456000809111011F928F938DEA95E02DC080916B
:104570001001262F30E0280F311D2F3F310524F484
:10458000680F6093100103C08FEF8093100180913A
:1045900010011F928F9384E995E016C080910F015E
:1045A000262F30E0280F311D2F3F310524F4680FEE
:1045B00060930F0103C08FEF80930F0180910F0173
:1045C0001F928F9389E795E09F938F930E945006E7
:1045D0000F900F900F900F900895833081F128F481
:1045E000813059F08230D1F00895853009F449C006
:1045F000B8F1863009F456C0089580911401681707
:1046000020F4861B8093140102C010921401809143
:1046100014011F928F938AE695E054C08091130194
:10462000681720F4861B8093130102C010921301B7
:10463000809113011F928F9388E595E043C080918C
:104640001201681720F4861B8093120102C0109299
:104650001201809112011F928F9385E495E032C080
:1046600080911101681720F4861B8093110102C00C
:1046700010921101809111011F928F9380E395E0B8
:1046800021C080911001681720F4861B80931001CF
:1046900002C010921001809110011F928F9387E148
:1046A00095E010C080910F01681720F4861B80935D
:1046B0000F0102C010920F0180910F011F928F9382
:1046C0008CEF94E09F938F930E9450060F900F9071
:1046D0000F900F900895CF93C82F1F928F9381E072
:1046E00098E09F938F930E94500681E090E0A0E0B5
:1046F000B0E0BC01CD0104C0660F771F881F991F71
:10470000CA95D2F70E944F1C0F900F900F900F90F8
:10471000CF910C944A18CF93873288F58E3108F0E8
:104720000BC18E3009F487C0D8F4873009F460C01B
:104730008B3009F44FC0863009F002C18091BE0170
:10474000817F8E7F8093BE0186E098E00E94B7054E
:104750008FEB9AE00E94B70581E08093CE0146C0BE
:10476000863109F4B0C020F4803109F47AC0E8C081
:10477000893109F491C08B3109F449C0E1C0883313
:1047800049F150F4893209F4D5C0853309F4D2C017
:10479000873209F0D5C0CEC0833409F4CBC028F4E9
:1047A0008A3308F4CDC08953C8C0883409F0C8C022
:1047B0000E944A188EEA9AE00E94B7052FEF83ED17
:1047C00090E3215080409040E1F700C000000E943B
:1047D000281F0CC08DE298E041C085E99AE00E9454
:1047E000B7058091BE0181608093BE01C1E0ADC07C
:1047F0008091BE01C82FC17080FFEFCF81EA9AE09F
:104800000E94B7058091BE01817F8E7F3FC090914D
:10481000BE0191FBCC27C0F981E0C827892FC0FBDE
:1048200081F98093BE01CC2319F088E89AE029C071
:104830008AE79AE013C09091BE0192FBCC27C0F9A1
:1048400081E0C827892FC0FB82F98093BE01CC2369
:1048500019F08BE69AE015C08BE59AE00E94B70547
:10486000C5CF9091BE0193FBCC27C0F981E0C8274A
:10487000892FC0FB83F98093BE01CC2351F08FE4D4
:104880009AE00E94B7058091BE0181608093BE01CD
:104890005CC082E49AE0E2CF83E39AE00E94B7052D
:1048A00080E19AE00E94B7058BEC99E00E94B70581
:1048B0008EE999E00E94B70589E599E00E94B70565
:1048C0008BE299E0CBCF8DE199E00E94B7050E9481
:1048D000C5111F928F9383E099E09F938F930E945D
:1048E000500680910C011F928F938CEE98E09F935D
:1048F0008F930E94500680915B011F928F9389EDE8
:1049000098E09F938F930E9450060E94CD1E9F9324
:104910008F937F936F9382EC98E09F938F930E9485
:1049200050068DB79EB742960FB6F8949EBF0FBE45
:104930008DBF5CCF80E001C08D510E946B2356CFAC
:1049400080EC98E00E94B705C0E08C2FCF910895CD
:1049500080E0089580E00895CF93C82F8091CE0124
:10496000813069F020F0823009F449C040C167E02D
:104970008FE00E944C13882309F43FC106C067E012
:104980008FE00E944C13882361F08C2F0E94A82492
:10499000811104C08C2F0E948B232FC081E090E0F6
:1049A0002CC08C2F0E94AA24811126C0C431E1F0B2
:1049B00070F4CB3081F0C031D1F40E94332289EF02
:1049C00097E00E94B70582E08093CE0115C0C932FE
:1049D00059F0C83361F486E098E00E94B7058DEF86
:1049E00097E00E94B70508C01092CE0104C187EF7E
:1049F00097E00E94B705FFC081E08170FEC0C4321D
:104A000028F5CE3108F0C1C0CB30A1F1D0F4C730C9
:104A100009F0D3C08EE18093140182E380931301E7
:104A20008AE08093120184E18093110188E08093F1
:104A3000100188E280930F018DE996E00E94B7058E
:104A4000BFC0C33149F1C431C1F0B7C0CB3409F4A0
:104A5000A9C028F4C93289F0C83361F0AEC0C135AD
:104A600009F49EC0C23509F499C0CE3409F0A5C03E
:104A70006AE09EC00E943322A3C08091CD018823AA
:104A800019F01092CD019CC08AEA96E00E94B70509
:104A900081E08093CE01B1C084E896E00E94B70522
:104AA00082E796E00E94B705809114011F928F93D0
:104AB0008FE696E09F938F930E9450068DE696E0D6
:104AC0000E94B7058BE596E00E94B705809113011F
:104AD0001F928F9388E596E09F938F930E945006D4
:104AE00086E596E00E94B70587E496E00E94B70548
:104AF000809112011F928F9384E496E09F938F938D
:104B00000E94500682E496E00E94B70581E396E099
:104B10000E94B705809111011F928F938EE296E05B
:104B20009F938F930E9450068CE296E00E94B705F7
:104B300087E196E00E94B705809110011F928F9344
:104B400084E196E09F938F930E94500682E196E065
:104B50000E94B7058BEF95E00E94B70580910F0189
:104B60001F928F9388EF95E09F938F930E9450063A
:104B700086EF95E00E94B7058DB79EB748960FB6B1
:104B8000F8949EBF0FBE8DBF1BC0CE51EC2FF0E03E
:104B9000E65DFE4F80818093CD0112C061E003C0CD
:104BA00061E006C06AE08091CD010E944A2208C0FF
:104BB0008091CD010E94ED2203C08BE996E013C0E5
:104BC0008091CD01882369F01F928F9385E996E04B
:104BD0009F938F930E9450060F900F900F900F900D
:104BE00004C082E996E00E94B70581E006C01092F9
:104BF000CE0180E002C080E000CFCF9108950E94F6
:104C000006266894B1110C94952608950E947A2680
:104C100088F09F5798F0B92F9927B751B0F0E1F07D
:104C2000660F771F881F991F1AF0BA95C9F714C02D
:104C3000B13091F00E949426B1E008950C9494262E
:104C4000672F782F8827B85F39F0B93FCCF3869566
:104C500077956795B395D9F73EF4909580957095C3
:104C600061957F4F8F4F9F4F0895E89409C097FB40
:104C70003EF490958095709561957F4F8F4F9F4F33
:104C80009923A9F0F92F96E9BB279395F695879577
:104C900077956795B795F111F8CFFAF4BB0F11F43A
:104CA00060FF1BC06F5F7F4F8F4F9F4F16C08823E1
:104CB00011F096E911C0772321F09EE8872F762F17
:104CC00005C0662371F096E8862F70E060E02AF058
:104CD0009A95660F771F881FDAF7880F9695879544
:104CE00097F9089557FD9058440F551F59F05F3FAD
:104CF00071F04795880F97FB991F61F09F3F79F0FE
:104D000087950895121613061406551FF2CF46957F
:104D1000F1DF08C0161617061806991FF1CF869501
:104D20007105610508940895E894BB2766277727E5
:104D3000CB0197F908950E94AE260C941F270E947C
:104D4000112738F00E94182720F0952311F00C94B9
:104D500008270C940E2711240C9495260E94722685
:104D600070F3959FC1F3950F50E0551F629FF001BE
:104D7000729FBB27F00DB11D639FAA27F00DB11DD7
:104D8000AA1F649F6627B00DA11D661F829F222760
:104D9000B00DA11D621F739FB00DA11D621F839FE7
:104DA000A00D611D221F749F3327A00D611D231FBD
:104DB000849F600D211D822F762F6A2F11249F570B
:104DC00050409AF0F1F088234AF0EE0FFF1FBB1F0E
:104DD000661F771F881F91505040A9F79E3F5105CD
:104DE00080F00C9408270C9495265F3FE4F3983EDE
:104DF000D4F3869577956795B795F795E7959F5F77
:104E0000C1F7FE2B880F911D9695879597F9089508
:104E100097F99F6780E870E060E008959FEF80EC6D
:104E2000089500240A941616170618060906089510
:104E300000240A9412161306140605060895092E76
:104E40000394000C11F4882352F0BB0F40F4BF2BE5
:104E500011F460FF04C06F5F7F4F8F4F9F4F089525
:104E6000991B79E004C0991F961708F0961B881FBC
:104E70007A95C9F78095089597FB072E16F400944C
:104E800007D077FD09D00E94562707FC05D03EF4D5
:104E9000909581959F4F0895709561957F4F0895E6
:104EA000EE0FFF1F0590F491E02D0994AA1BBB1B88
:104EB00051E107C0AA1FBB1FA617B70710F0A61B1A
:104EC000B70B881F991F5A95A9F780959095BC013B
:084ED000CD010895F894FFCF15
:104ED800FFFF2A0A1B0BF80AC40A900A01B401282A
:104EE80008140A321E404D36221A04CD0397037562
:104EF8000301031A0333034C0300010203040506EC
:044F0800070809008D
:106800000000EA44E944E2440400050006000700F1
:10681000080009000A000B000C000D000E000F001C
:1068200010001100120013001400150016001700CC
:10683000180019001A001B001C001D001E001F007C
:10684000200021002200230024002500260027002C
:10685000280029002A002B002C002D002E002F00DC
:10686000300031A132003300340035A1360037004A
:10687000380082003A003B003C003D003E003F00F3
:1068800040004100420043004400450046004700EC
:10689000480049004A004B004C004D004E004F009C
:1068A000500051005200530067005400550056003C
:1068B000580059005A005B005C005D005E005F00FC
:1068C0006000610062006300640000005700000087
:1068D000CD440000000000000000000000000000A7
:1068E0000000000000007300000000000000000035
:1068F000E000E100E200E300E400E500E600E7007C
:106900000100010001000100EA4401000100E2442D
:106910000100010001000100460001004A004B0097
:10692000010001004700480001000100E9440100A6
:106930000100010001000100010001003A003B00DC
:106940003C003D003E003F0040004100420043004B
:10695000010001004C00010001004400450052000C
:1069600049000100010050004F0001004D004E00A1
:1069700051000100010001000100010001000100BF
:1069800001000100010001000100010001000100FF
:1069900001000100010001000100010001004D00A3
:1069A0004A004E004B0001000100010001000100FF
:1069B00001000100010001000100010001000100CF
:1069C00001000100010001000100010001000100BF
:1069D00001000100010001000100010001000100AF
:1069E000010001000100010001000100010001009F
:1069F000010001000100010001000100010001008F
:00000001FF
